:1000000010C017C016C015C014C013C012C011C054
:1000100010C00FC00EC00DC00CC00BC00AC009C07C
:1000200008C011241FBECFE5D1E0DEBFCDBF02D096
:10003000C6C0E6CF80E886BD16BCDE98D69ADF98AB
:10004000D79A80E08E31A8F4DE9ADF9AE7E8F3E1F0
:100050003197F1F700C00000DE98DF98FFED28E24D
:1000600031E0F15020403040E1F700C000008F5FE8
:10007000E9CF8EE1DE9ADF9AEBE4FDE13197F1F70B
:1000800000C00000DE98DF98FFE021E231E0F1508F
:1000900020403040E1F700C00000815059F78EE168
:1000A000DE9ADF9AEFE0F7E23197F1F700C0000047
:1000B000DE98DF98FFE329E131E0F1502040304045
:1000C000E1F700C00000815059F78EE1DE9AE7E8C1
:1000D000F3E13197F1F700C00000DE98FFED28E270
:1000E00031E0F15020403040E1F700C00000815085
:1000F00069F78EE1DF9AE7E8F3E13197F1F700C0A5
:100100000000DF98FFED28E231E0F1502040304060
:10011000E1F700C00000815069F78EE1DE9AEBE460
:10012000FDE13197F1F700C00000DE98FFE021E229
:1001300031E0F15020403040E1F700C00000815034
:1001400069F78EE1DF9AEBE4FDE13197F1F700C04A
:100150000000DF98FFE021E231E0F1502040304024
:10016000E1F700C00000815069F78EE1DE9AEFE010
:10017000F7E23197F1F700C00000DE98FFE329E1D4
:1001800031E0F15020403040E1F700C000008150E4
:1001900069F78EE1DF9AEFE0F7E23197F1F700C0FF
:1001A0000000DF98FFE329E131E0F15020403040CA
:1001B000E1F700C00000815069F780E045CFF89476
:0201C000FFCF6F
:00000001FF
